** EXPERIMENTAL (HLL) ** Open Watcom Linker Version 1.6beta1 Limited Availability
Portions Copyright (c) 1985-2002 Sybase, Inc. All Rights Reserved.
Created on:       13/11/17 16:27:53
Warning! W1121: file U:/tmp\ldconv__localemodule_obj_2b9852885ae0154790.obj(U:\DEV\python-2.7.5\Modules\_localemodule.c): '_init_locale' has already been exported
Executable Image: build/lib.os2knix-2.7/_locale.pyd
creating an OS/2 EMX dynamic link library


                        +------------+
                        |   Groups   |
                        +------------+

Group                           Address              Size
=====                           =======              ====

CGROUP                          0001:00000000        00006c40
DGROUP                          0002:00000000        000008c0



                        +--------------+
                        |   Segments   |
                        +--------------+

Segment                Class          Group          Address         Size
=======                =====          =====          =======         ====

TEXT32                 CODE           CGROUP         0001:00000000   00006c40
________TEXT           CODE           CGROUP         0001:00006c40   00000000
DATA32                 DATA           DGROUP         0002:00000000   000005e0
SET1__os2dll           DATA           DGROUP         0002:000005e0   00000004
SET2__os2dll           DATA           DGROUP         0002:000005e4   00000000
SET3__os2dll           DATA           DGROUP         0002:000005e4   00000004
SET1___CTOR_LIST__     DATA           DGROUP         0002:000005e8   00000004
SET2___CTOR_LIST__     DATA           DGROUP         0002:000005ec   00000004
SET3___CTOR_LIST__     DATA           DGROUP         0002:000005f0   00000004
SET1___DTOR_LIST__     DATA           DGROUP         0002:000005f4   00000004
SET2___DTOR_LIST__     DATA           DGROUP         0002:000005f8   00000000
SET3___DTOR_LIST__     DATA           DGROUP         0002:000005f8   00000004
SET1___crtinit1__      DATA           DGROUP         0002:000005fc   00000004
SET2___crtinit1__      DATA           DGROUP         0002:00000600   00000000
SET3___crtinit1__      DATA           DGROUP         0002:00000600   00000004
SET1___crtexit1__      DATA           DGROUP         0002:00000604   00000004
SET2___crtexit1__      DATA           DGROUP         0002:00000608   00000000
SET3___crtexit1__      DATA           DGROUP         0002:00000608   00000004
SET1___eh_frame__      DATA           DGROUP         0002:0000060c   00000004
SET2___eh_frame__      DATA           DGROUP         0002:00000610   00000008
SET3___eh_frame__      DATA           DGROUP         0002:00000618   00000004
SET1___eh_init__       DATA           DGROUP         0002:0000061c   00000004
SET2___eh_init__       DATA           DGROUP         0002:00000620   00000004
SET3___eh_init__       DATA           DGROUP         0002:00000624   00000004
SET1___eh_term__       DATA           DGROUP         0002:00000628   00000004
SET2___eh_term__       DATA           DGROUP         0002:0000062c   00000004
SET3___eh_term__       DATA           DGROUP         0002:00000630   00000004
SET1___fork_parent1__  DATA           DGROUP         0002:00000634   00000004
SET2___fork_parent1__  DATA           DGROUP         0002:00000638   00000000
SET3___fork_parent1__  DATA           DGROUP         0002:00000638   00000004
SET1___fork_child1__   DATA           DGROUP         0002:0000063c   00000004
SET2___fork_child1__   DATA           DGROUP         0002:00000640   00000000
SET3___fork_child1__   DATA           DGROUP         0002:00000640   00000004
________DATA           DATA           DGROUP         0002:00000650   00000000
BSS32                  BSS            DGROUP         0002:00000650   00000140
c_common               BSS            DGROUP         0002:00000790   00000130
________BSS            BSS            DGROUP         0002:000008c0   00000000


                        +----------------+
                        |   Memory Map   |
                        +----------------+

* = unreferenced symbol
+ = symbol only referenced locally

Address        Symbol
=======        ======

Module: U:\usr\lib\dll0hi.obj({standard input})
0001:00000000* __text
0002:00000000* __data
0002:00000000* ___data_start
0002:00000650* ___bss_start
0002:000005e0+ __os2dll
0002:000005e8  ___CTOR_LIST__
0002:000005f4  ___DTOR_LIST__
0002:000005fc* ___crtinit1__
0002:00000604* ___crtexit1__
0002:0000060c  ___eh_frame__
0002:0000061c  ___eh_init__
0002:00000628  ___eh_term__
0002:00000634+ ___fork_parent1__
0002:0000063c+ ___fork_child1__
Module: U:/tmp\ldconv__localemodule_obj_2b9852885ae0154790.obj(U:\DEV\python-2.7.5\Modules\_localemodule.c)
0001:000011e4  _init_locale
Module: U:\usr\local473\lib\libc_dll.lib(dllinit.obj)
0001:000018a0  _DLL_InitTerm
Module: U:\usr\lib\libend.lib(src/libend/386/endlink386.asm)
0002:000008c0  _end
0002:00000650  _edata
Module: U:\usr\lib\libend.lib(src/libend/386/end.asm)
0001:00006c40* _etext
0001:00006c40* __etext
0000:00000000  WEAK$ZERO
0002:000008c0  __end
0002:00000650  __edata
Module: U:\extras\lib\intl.lib(intl-compat.obj)
0001:00001900* _gettext
0001:00001910* _dgettext
0001:00001920  _dcgettext
0001:00001930* _ngettext
0001:00001940* _dngettext
0001:00001950* _dcngettext
0001:00001960  _textdomain
0001:00001970  _bindtextdomain
0001:00001980  _bind_textdomain_codeset
Module: U:\tmp\ldconv_libgcc_so_d_a_2b9852885ae1135f48.lib(emx-ctordtor.obj)
0001:00001990  ___ctordtorInit
0001:000019c4  ___ctordtorTerm
Module: U:\extras\lib\intl.lib(gettext.obj)
0001:00001a00  _libintl_gettext
Module: U:\extras\lib\intl.lib(dgettext.obj)
0001:00001a30  _libintl_dgettext
Module: U:\extras\lib\intl.lib(dcgettext.obj)
0001:00001a60  _libintl_dcgettext
Module: U:\extras\lib\intl.lib(ngettext.obj)
0001:00001aa0  _libintl_ngettext
Module: U:\extras\lib\intl.lib(dngettext.obj)
0001:00001ae0  _libintl_dngettext
Module: U:\extras\lib\intl.lib(dcngettext.obj)
0001:00001b20  _libintl_dcngettext
Module: U:\extras\lib\intl.lib(textdomain.obj)
0001:00001b60  _libintl_textdomain
Module: U:\extras\lib\intl.lib(bindtextdom.obj)
0001:00001c10  _libintl_bindtextdomain
0001:00001c40  _libintl_bind_textdomain_codeset
Module: U:\tmp\ldconv_libgcc_so_d_a_2b9852885ae1135f48.lib(emx-eh.obj)
0001:00001fa0  ___ehInit
0001:00001fd6* ___ehTerm
Module: U:\extras\lib\intl.lib(dcigettext.obj)
0002:00000790  _libintl_nl_domain_bindings
0001:00002010  _libintl_nl_default_default_domain
0001:00002220  _libintl_dcigettext
0001:000027d0  __nl_find_msg
0002:000005b0  _libintl_nl_current_default_domain
Module: U:\tmp\ldconv_libgcc_a_2b9852885ae015dfe8.lib(_alloca.obj)
0001:00002d50  __alloca
Module: U:\extras\lib\intl.lib(finddomain.obj)
0001:00002d80  __nl_find_domain
Module: U:\extras\lib\intl.lib(osdep.obj)
0002:000007a0  _libintl_nl_default_dirname
0001:00002fa0  __nl_getenv
0002:000006b0* __nlos2_libdir
0002:000006b4  __nlos2_localealiaspath
0002:000006b8* __nlos2_localedir
Module: U:\extras\lib\intl.lib(log.obj)
0001:00003230  __nl_log_untranslated
Module: U:\extras\lib\intl.lib(hash-string.obj)
0001:00003690  _libintl_hash_string
Module: U:\extras\lib\intl.lib(loadmsgcat.obj)
0002:000008b0  __nl_msg_cat_cntr
0001:000036e0  __nl_load_domain
Module: U:\extras\lib\intl.lib(localename.obj)
0001:00004ab0  __nl_locale_name_posix
0001:00004b10  __nl_locale_name_default
0001:00004b20* __nl_locale_name
Module: U:\extras\lib\intl.lib(langprefs.obj)
0001:00004b80  __nl_language_preferences_default
Module: U:\extras\lib\intl.lib(l10nflist.obj)
0001:00004b90  __nl_make_l10nflist
0001:000050b0  __nl_normalize_codeset
Module: U:\extras\lib\intl.lib(localealias.obj)
0001:00005210  __nl_expand_alias
Module: U:\extras\lib\intl.lib(explodename.obj)
0001:00005830  __nl_explode_name
Module: U:\extras\lib\intl.lib(plural-exp.obj)
0001:00005a20  _libintl_gettext_extract_plural
0002:000005c0* _libintl_gettext_germanic_plural
Module: U:\extras\lib\intl.lib(relocatable.obj)
0001:00005b20* _libintl_set_relocation_prefix
0001:00005bf0  _libintl_relocate
Module: U:\extras\lib\intl.lib(plural.obj)
0001:00005ed0  _libintl_gettextparse
0001:000068a0* _libintl_gettext_free_exp
Error! E3008: cannot open build/lib.os2knix-2.7/_locale.pyd : Permission denied
